:10000000D7288030A100FE3091200130912075303A
:10001000A6003030A228A101A117AE00FE30912029
:100020002E089128A401A900AA01A01124080319EF
:10003000A0150530A3002730A80010302B20033076
:10004000A800E8302B20A80164302B20A8010A303A
:100050002B2029083228A7002A08A6002908A50075
:10006000B6202508A500A3030319A011240803192D
:100070003C282302031843282508031DA011A019BA
:100080004328303E91280800AC00061186118316E3
:10009000061186110F30860583122C08A0186E28D1
:1000A0003E30A6008030A2203330AB0082201330D7
:1000B000A6008830A22082206430A12082206430F3
:1000C000A1202230AB00822028306D200C306D2022
:1000D00006306D20A0142C086E282014AB00201CC4
:1000E0007C288611033C031C812881200730A60050
:1000F000D030A220031408002014FE3C03198F28DE
:100100008615201C201006150F3086052B08F039A7
:1001100086040611AB0E201882283230A1202C084C
:10012000D228A11B44280800A801A700FF30A70778
:10013000031CA807031CD2280330A600DF30A2202E
:100140009628A601E83EA500A609FC30031CAB28B2
:10015000A5070318A828A5070000A60FA82825189A
:10016000B128A51CB5280000B5280800AA01A901DE
:100170001030AB00260DA90DAA0D2708A9022808EA
:10018000031C280FAA020318CC282708A90728084F
:100190000318280FAA070310A50DA60DAB0BBA284C
:1001A0002508D22883138312031300000800A0013E
:1001B000AF01B001B10101200130A800F430952059
:1001C0008030A10080300B20433044202030442078
:1001D000453044206C304420653044206B3044204E
:1001E0008030A100C0300B205330442074304420B4
:1001F000793044206E3044207530442073304420E0
:100200000330A800E83095208030A10080300B201A
:100210002030442044204420442044204420803086
:10022000A100C0300B202030442044204420442032
:10023000442044208030A100C0300B2030304420C6
:10024000203044203A3044203030442020304420B4
:100250003A3044203030442044202E298030A10000
:1002600080300B204F304420463044204420061C70
:10027000452932309420061C3E2939290618452983
:10028000831605118312051546292E298030A100F9
:1002900080300B204F3044204E304420203044200A
:1002A000061C612932309420061C5729542906184F
:1002B00061298316051183120511AF01B001B10147
:1002C0002E2903309420AF0A64302F02031D6A29BF
:1002D000AF01B00A3C303002031D7029B001B10AF1
:1002E0008030A100C0300B202030442044203A3020
:1002F00044202030442044203A3044208030A10063
:10030000C0300B20310812208030A100C3300B20F8
:10031000300812208030A100C6300B202F08122098
:0603200050296300912941
:02400E00703F01
:00000001FF
